:020000040000FA
:100000001D2929345334283488010B11C30F0532BC
:10001000C40F0332C50F0132C216C80F0332C9081C
:10002000031DC903B008031DB40B0432B0033D081F
:10003000B400C217B208031DB60B0432B2033D0868
:10004000B6004217B108031DB50B0832FF1D02327E
:10005000B1010332B1033F08B500C217B308031D55
:10006000B70B0900FF1D0232B3010332B3033F088F
:10007000B7004217090004341434083464340A34D5
:100080002934533428340B00000002340634083479
:1000900004340B00000001340534073403340B0032
:1000A00001340234043408341034203440348034B1
:1000B0000B000134033407340F341F343F347F34D2
:1000C000FF342920532028206400031D0532B90184
:1000D000BA01BB01BC010800B90019303902031C88
:1000E00007325820BC00FF30BB00BA00B90008003E
:1000F000BC0111303902031C06325820BB00FF300E
:10010000BA00B9000800BC01BB0109303902031C68
:1001100005325820BA00FF30B9000800BC01BB010D
:10012000BA0139035820B900080064000319CF331D
:10013000B90019303902031C06324F20BC00BB0144
:10014000BA01B9010800BC0111303902031C0532A3
:100150004F20BB00BA01B9010800BC01BB01093046
:100160003902031C04324F20BA00B9010800BC0157
:10017000BB01BA0139034F20B90008001030B900A3
:1001800022008C1222008C102000C735C60D2200E0
:1001900003180C14031C0C10640000008C142000C5
:1001A000B90BF03322008C168C10200008000430AC
:1001B000BA003A081F3E84000008C7003A084320EE
:1001C000C600BE20BA0BF53308000430BA003A0866
:1001D000233E84000008C7003A084920C600BE201C
:1001E000BA0BF5330800C801C81EFE330800421CD4
:1001F000933242108B132300FF30910005309200A0
:1002000015131516151555309600AA30960095143D
:100210000000000015111513151595167F089300A1
:1002200034309400951255309600AA3096009514FB
:1002300000000000151120006F3222008C162100F2
:1002400073309900DC308C00FF308E00D8309E0077
:100250009F015430950091019201930189309D00D6
:10026000D0309700230014308C008E012400C83059
:100270008C008E012A00EC3091009500200098013E
:100280009C0120308B008501C201FA30C500C401F9
:10029000C3013B20BD007A30C1003C20BE0040308D
:1002A0000A00C1073D20BF0041300A00C1073E20BF
:1002B000C00042300A00C1071E30C10203193F20AE
:1002C000C1005C30FF0001300A00FF0702300A0065
:1002D000FF0703300A00FF0703190232FF30FF0057
:1002E0007F0385310A008031FF00FF30C600C7015F
:1002F000BE20FC30C6000130C700BE20F930C60069
:10030000C701BE20FB30C6000730C700BE20FA3050
:10031000C6000F30C700BE201E30B100B300B001D0
:10032000B201C21742178B1720008C19E12AF32063
:100330000130A000A101A201A301D7207F1805323E
:10034000FF30A400A500A6000332A401A501A60168
:100350000130A700E52064008C1DFD33F32005303B
:10036000C900C9080319F72864008C19FA33F3206F
:100370000230C900C9080319053264008C1DFA3324
:10038000F3202532C801C2140430C900C81F053249
:10039000A401A501A601A70108327F180432FF308D
:1003A000A400A500A6000130A700E5206400C21C3F
:1003B00004328C1DE933F320C210C9080319B83385
:1003C0008C19E433F3200130FF064214DB33023092
:1003D000A000A101A201A301D720FF180632AA3074
:1003E000A400A500A600A70008322030A700043012
:1003F000A6000430A5002530A400E5200530C90082
:10040000C9080319F72864008C19FA33F320023065
:10041000C900C9080319053264008C1DFA33F320A2
:100420003032C801C2140430C900C81F0532A4010B
:10043000A501A601A7011332FF180632AA30A400B5
:10044000A500A600A7000B322030A70029300430F9
:10045000A60053300430A50028302530A400E52044
:100460006400C21C04328C1DDE33F320C210C908A4
:100470000319AD338C19D933F3200230FF0642142F
:10048000D0330430A000A101A201A301D7207F191D
:100490000632FF30A400A500A601A7010632FF30F6
:1004A000A400A500A6010130A700E5200530C90081
:1004B000C9080319F72864008C19FA33F3200230B5
:1004C000C900C9080319053264008C1DFA33F320F2
:1004D0002B32C801C2140430C900C81F0532A40160
:1004E000A501A601A7010E327F190632FF30A40034
:1004F000A500A601A7010632FF30A400A500A601B1
:100500000130A700E5206400C21C04328C1DE333D7
:10051000F320C210C9080319B4338C19DE33F32059
:100520000430FF064214D5330830A000A101A20117
:10053000A301D720FF1904321130A400A500023214
:10054000A401A5010130A600A701E5200530C900DE
:10055000C9080319F72864008C19FA33F320023014
:10056000C900C9080319053264008C1DFA33F32051
:100570009829C801C2140430C900C81F0532A4015B
:10058000A501A601A7010B32FF1904321130A40006
:10059000A5000232A401A5010130A600A701E520B3
:1005A0006400C21C04328C1DE633F320C210C9085B
:1005B0000319BA338C19E133F3200830FF064214D3
:1005C000D83364002000C21B6832421B4332210032
:1005D0009D18942909301D1D0D309D002000863185
:1005E000FF1C883121009C180A141C361B0C2000AB
:1005F0000A008031B80021009D141D191632200018
:1006000038083002031894293808B0003E08B400B6
:1006100041083802031C413231083802031C3D32C4
:100620003808B1004008B5003832200038083202DE
:10063000031894293808B2003E08B6004108380271
:10064000031C083233083802031C04323808B30094
:100650004008B7004213C21E7F1DB3013308952026
:100660003908AC003A08AD003B08AE003C08AF00CA
:100670003208C21E7F1802326420013295203908E8
:100680002C04A4003A082D04A5003B082E04A60063
:100690003C082F04A700E5209429C213C21E7F1D29
:1006A000B101310895203908A8003A08A9003B0893
:1006B000AA003C08AB003008C21E7F18023264203A
:1006C0000132952039082804A0003A082904A10025
:1006D0003B082A04A2003C082B04A300D72094293D
:040BFC000234063485
:100C00000034003400340034003400340034003444
:100C10000134023403340334043404340534053419
:100C200006340634063407340734073408340834ED
:100C3000083409340934093409340A340A340A34CA
:100C40000A340B340B340B340B340B340C340C34AB
:100C50000C340C340C340C340D340D340D340D3490
:100C60000D340D340D340E340E340E340E340E3477
:100C70000E340E340E340F340F340F340F340F345F
:100C80000F340F340F340F34103410341034103448
:100C90001034103410341034103410341034113433
:100CA000113411341134113411341134113411341C
:100CB0001134113411341234123412341234123407
:100CC00012341234123412341234123412341234F4
:100CD00013341334133413341334133413341334DC
:100CE00013341334133413341334133413341334CC
:100CF00013341434143414341434143414341434B5
:100D000014341434143414341434143414341434A3
:100D1000143414341434143415341534153415348F
:100D2000153415341534153415341534153415347B
:100D3000153415341534153415341534153415346B
:100D40001534153416341634163416341634163455
:100D50001634163416341634163416341634163443
:100D60001634163416341634163416341634163433
:100D70001634163416341634163417341734173420
:100D8000173417341734173417341734173417340B
:100D900017341734173417341734173417341734FB
:100DA00017341734173417341734173417341734EB
:100DB00017341734173418341834183418341834D6
:100DC00018341834183418341834183418341834C3
:100DD00018341834183418341834183418341834B3
:100DE00018341834183418341834183418341834A3
:100DF0001834183418341834183419341934193490
:100E0000193419341934193419341934193419347A
:100E1000193419341934193419341934193419346A
:100E2000193419341934193419341934193419345A
:100E3000193419341934193419341934193419344A
:100E400019341934193419341A341A341A341A3436
:100E50001A341A341A341A341A341A341A341A3422
:100E60001A341A341A341A341A341A341A341A3412
:100E70001A341A341A341A341A341A341A341A3402
:100E80001A341A341A341A341A341A341A341A34F2
:100E90001A341A341A341A341A341A341A341A34E2
:100EA0001B341B341B341B341B341B341B341B34CA
:100EB0001B341B341B341B341B341B341B341B34BA
:100EC0001B341B341B341B341B341B341B341B34AA
:100ED0001B341B341B341B341B341B341B341B349A
:100EE0001B341B341B341B341B341B341B341B348A
:100EF0001B341B341B341B341B341B341B341B347A
:100F00001B341B341C341C341C341C341C341C3463
:100F10001C341C341C341C341C341C341C341C3451
:100F20001C341C341C341C341C341C341C341C3441
:100F30001C341C341C341C341C341C341C341C3431
:100F40001C341C341C341C341C341C341C341C3421
:100F50001C341C341C341C341C341C341C341C3411
:100F60001C341C341C341C341C341C341C341C3401
:100F70001C341C341D341D341D341D341D341D34EB
:100F80001D341D341D341D341D341D341D341D34D9
:100F90001D341D341D341D341D341D341D341D34C9
:100FA0001D341D341D341D341D341D341D341D34B9
:100FB0001D341D341D341D341D341D341D341D34A9
:100FC0001D341D341D341D341D341D341D341D3499
:100FD0001D341D341D341D341D341D341D341D3489
:100FE0001D341D341D341D341D341D341D341D3479
:100FF0001D341D341E341E341E341E341E341E3463
:101000000034003400340034003400340034003440
:10101000003400340134013401340134013401342A
:101020000134013401340134013401340134013418
:101030000134013401340234023402340234023403
:1010400002340234023402340234023402340234F0
:1010500002340234023402340334033403340334DC
:1010600003340334033403340334033403340334C8
:1010700003340334033403340334043404340434B5
:1010800004340434043404340434043404340434A0
:10109000043404340434043404340434053405348E
:1010A0000534053405340534053405340534053478
:1010B0000534053405340534053405340534063467
:1010C0000634063406340634063406340634063450
:1010D0000634063406340634063406340634063440
:1010E0000734073407340734073407340734073428
:1010F0000734073407340734073407340734073418
:101100000734083408340834083408340834083400
:1011100008340834083408340834083408340834EF
:1011200008340834093409340934093409340934D9
:1011300009340934093409340934093409340934C7
:101140000934093409340A340A340A340A340A34B2
:101150000A340A340A340A340A340A340A340A349F
:101160000A340A340A340A340B340B340B340B348B
:101170000B340B340B340B340B340B340B340B3477
:101180000B340B340B340B340B340C340C340C3464
:101190000C340C340C340C340C340C340C340C344F
:1011A0000C340C340C340C340C340C340D340D343D
:1011B0000D340D340D340D340D340D340D340D3427
:1011C0000D340D340D340D340D340D340D340E3416
:1011D0000E340E340E340E340E340E340E340E34FF
:1011E0000E340E340E340E340E340E340E340E34EF
:1011F0000F340F340F340F340F340F340F340F34D7
:101200000F340F340F340F340F340F340F340F34C6
:101210000F341034103410341034103410341034AF
:10122000103410341034103410341034103410349E
:101230001034103411341134113411341134113488
:101240001134113411341134113411341134113476
:101250001134113411341234123412341234123461
:10126000123412341234123412341234123412344E
:10127000123412341234123413341334133413343A
:101280001334133413341334133413341334133426
:101290001334133413341334133414341434143413
:1012A00014341434143414341434143414341434FE
:1012B00014341434143414341434143415341534EC
:1012C00015341534153415341534153415341534D6
:1012D00015341534153415341534153415341634C5
:1012E00016341634163416341634163416341634AE
:1012F000163416341634163416341634163416349E
:101300001734173417341734173417341734173485
:101310001734173417341734173417341734173475
:10132000173418341834183418341834183418345E
:10133000183418341834183418341834183418344D
:101340001834183419341934193419341934193437
:101350001934193419341934193419341934193425
:101360001934193419341A341A341A341A341A3410
:101370001A341A341A341A341A341A341A341A34FD
:101380001A341A341A341A341B341B341B341B34E9
:101390001B341B341B341B341B341B341B341B34D5
:1013A0001B341B341B341B341B341C341C341C34C2
:1013B0001C341C341C341C341C341C341C341C34AD
:1013C0001C341C341C341C341C341C341D341D349B
:1013D0001D341D341D341D341D341D341D341D3485
:1013E0001D341D341D341D341D341D341D341E3474
:1013F0001E341E341E341E341E341E341E341E345D
:020000040001F9
:0600000029005300280056
:02000E001C0FC5
:02001000FB1CD7
:00000001FF
